:1000000012C02CC02BC02AC0D8C428C027C026C00C
:1000100025C024C023C022C021C020C01FC01EC0D4
:100020001DC01CC01BC011241FBECFE5D4E0DEBF25
:10003000CDBF10E0A0E6B0E0EAEFFFE002C005901F
:100040000D92AA36B107D9F711E0AAE6B0E001C0D7
:100050001D92A538B107E1F772D4CDC7D1CFAC015D
:100060008091B400873219F481E08093B3008091CD
:10007000B400882351F487EB90E09093B60080930E
:10008000B50087E28093B4000EC08091B400815027
:100090008093B4008091B5009091B6000296909341
:1000A000B6008093B500E091B500F091B6005183A1
:1000B00040838091B300882309F1A0E020E030E084
:1000C00067EB70E0B1E0FB01E20FF31F80819181EB
:1000D000841B950B8F3C910544F480819181FA013A
:1000E000E81BF90BE836F1050CF0AB2F2E5F3F4F04
:1000F0002035310541F78A2FA11181E00895CF9372
:10010000DF93EC01ACDF882351F48CE0CC33D807CB
:1001100030F480E0C855D44018F081E001C080E0A0
:10012000DF91CF9108959C018BE02D36380788F43C
:100130001092B200E2E3F0E08081886080838081E9
:100140008F7E8083662329F4E8E3F0E08081806479
:1001500080838BE0253D380790F082E08093B200E9
:10016000E2E3F0E08081877F80838081806180830B
:10017000662329F4E8E3F0E08081806480838CE0EA
:100180002C33380790F081E08093B200E2E3F0E096
:100190008081877F8083808180618083662329F4CA
:1001A000E8E3F0E08081806480832F5B344078F462
:1001B000662329F4E8E3F0E080818F7B8083E2E32B
:1001C000F0E080818061808380818860808380917D
:1001D000B2000895DF92EF92FF920F931F93FC01FC
:1001E000D62E4817590768F4662329F4E8E3F0E0AF
:1001F000808180648083E2E3F0E080818F7E808371
:1002000032C08091AF00882321F081508093AF00ED
:1002100003C084E18093AF00BF01621B730B80E0D9
:1002200090E0A3D5A80197010AD673D52091AF001D
:10023000621768F4DD2029F4E8E3F0E080818F7B29
:100240008083E2E3F0E08081806180830CC0DD2068
:1002500029F4E8E3F0E0808180648083E2E3F0E069
:1002600080818F7E80831F910F91FF90EF90DF90B0
:100270000895EF92FF920F931F938C01F62E81EC5D
:1002800095E0841B950B0817190710F41092B00025
:1002900089E096E0841B950B8017910740F481E07C
:1002A0008093B000E2E3F0E08081877F808382EA80
:1002B00095E0841B950B0817190728F4E2E3F0E09A
:1002C000808188608083B80180E090E04ED524EA88
:1002D00033EF47E954E4AFD5181694F4C8016F2DF5
:1002E00048EE54E02FEB34E00F2EFFE0EF2EF0E865
:1002F000FF2EF8EF0F2FFEE31F2FF02D6BDF0CC04A
:10030000FF2029F4E8E3F0E080818F7B8083E2E343
:10031000F0E08081806180838091B0001F910F9117
:10032000FF90EF900895EF92FF920F931F938C012F
:10033000F62E9A01220F331F8DE69BE0821B930B52
:100340000817190710F41092B10089EE9BE0821B88
:10035000930B8017910740F481E08093B100E2E3B2
:10036000F0E08081877F808382EA95E0841B950B93
:10037000880F991F0817190728F4E2E3F0E080813D
:1003800088608083B80180E090E0EFD42BEF39EAF9
:1003900046E155E450D5181694F4C8016F2D41ED8F
:1003A00059E02AE639E00F2EFCECEF2EFCECFF2E94
:1003B000F6E40F2FFEE31F2FF02D0CDF0CC0FF2003
:1003C00029F4E8E3F0E080818F7B8083E2E3F0E0D2
:1003D0008081806180838091B1001F910F91FF9097
:1003E000EF900895EF92FF921F93CF93DF93162F14
:1003F0007A01A0E0B0E0BC01CD01B7D42DEF39E522
:100400004EEC50E41CD585D4DC01CB01EC0177DE49
:10041000882391F088E0CD30D80738F0CE01612FE5
:10042000A70181DF809307010CC0CE01612FA701D6
:1004300020DF8093070105C0CE01612F74DE809319
:10044000070180910701DF91CF911F91FF90EF90FD
:1004500008959C0180916E00882351F48DE1809372
:100460006E0083E790E09093700080936F000EC061
:1004700080916E00815080936E0080916F0090910A
:10048000700002969093700080936F00E0916F006F
:10049000F09170003183208340E050E020E030E0B4
:1004A00063E770E0FB01E20FF31F80819181481741
:1004B000590714F4408151812E5F3F4F2C33310591
:1004C00089F78FEA90E09093720080937100CA01DF
:1004D00005978734910514F086E490E09C019923F8
:1004E00014F420E030E086E4821B0895662331F0A6
:1004F000E8E3F0E08081806880830895AADF80933C
:10050000600080916000863431F4E8E3F0E080819F
:1005100080688083089580916C008823C9F480915D
:100520006B00882341F0E8E3F0E080818F778083DF
:1005300010926B0008C0E8E3F0E08081806880835F
:1005400081E080936B008091600080936C0005C017
:1005500080916C00815080936C0080916C00409180
:10056000600020916D0090E0840F911D30E028170D
:10057000390754F480916C009091600020916D00D7
:10058000980F921B90936C008091600080936D0097
:1005900080916C0080916C00873418F086E4809321
:1005A0006C00089580916A00882389F4B69B06C088
:1005B000E8E3F0E080818F7B808305C0E8E3F0E032
:1005C00080818064808384E180936A0008958150F3
:1005D00080936A000895DF93CF9300D000D0CDB709
:1005E000DEB7AC01662309F0D6C0863991050CF060
:1005F000D2C0009709F4CFC080910A01882309F086
:10060000CAC080911001909111019A01281B390BE9
:100610003A83298350931101409310018091630024
:100620009091640020910E0130910F01821B930B79
:100630009C838B83809163009091640090930F0161
:1006400080930E018B819C81181619062CF48981E8
:100650009A811816190644F08B819C81992304F520
:1006600089819A819923E4F484E090E09093620078
:100670008093610080910D01882319F084E08093BC
:100680000B0181E080930C0110920D0180910B0110
:10069000882331F082E090E09093620080936100C3
:1006A0008B819C8199232CF489819A8118161906D3
:1006B0004CF08B819C811816190604F589819A816A
:1006C0009923E4F48CEF9FEF909362008093610094
:1006D00080910C01882319F084E080930B0181E064
:1006E00080930D0110920C0180910B01882331F051
:1006F0008EEF9FEF909362008093610080910B01D9
:10070000882329F080910B01815080930B01809107
:100710006300909164002091610030916200280F85
:10072000391F30936400209363008091630090919F
:1007300064008B3F910564F08AEF90E09093640031
:10074000809363008CEF9FEF909362008093610031
:100750008091630090916400449764F484E190E098
:10076000909364008093630084E090E09093620033
:10077000809361008091610090916200880F991FC1
:100780009093620080936100809163009091640077
:100790009BBD8ABD30C06230B1F4809163009091FE
:1007A0006400CE9764F08091630090916400992377
:1007B0000CF40196959587959BBD8ABD06C08EE188
:1007C00090E09BBD8ABD613019F0463951059CF01F
:1007D0004837510564F084E190E090936400809381
:1007E000630084E090E090936200809361008EE16A
:1007F00090E09BBD8ABD4630510554F480910801BC
:10080000883C30F4809108018F5F8093080102C01A
:1008100010920801809108018F3B68F080910A01D5
:10082000882349F480910901882329F48FEF80936C
:100830000A018093090180910A01882359F0E7E3B6
:10084000F0E080818D7F808380910A0181508093C8
:100850000A010EC080910901882329F080910901C5
:10086000815080930901E7E3F0E08081826080831A
:100870000F900F900F900F90CF91DF910895829974
:1008800004C080E090E060E096D380E090E086D302
:100890008093840181E090E089D30895A7E3B0E0DC
:1008A0008C9182608C93E1E3F0E0808188608083AA
:1008B0008081806180838C9180648C938C9180682E
:1008C0008C93E5E3F0E080818860808380818061A3
:1008D0008083E2E3F0E080818460808380E888B9EF
:1008E00081E88FBD89E08EBD8EE190E09BBD8ABD21
:1008F00086E085BDE6E2F0E085EC808384E487B99C
:10090000808180648083808186FDFDCF84B185B144
:100910002EE088E190E00FB6F894A89581BD0FBE57
:1009200021BD80E489BFABDF909383018093820176
:10093000E5E5F0E080818068808378940895AEDFFB
:10094000E5E5F0E0A89580818068808388958081C6
:100950008F778083F7CF0F931F939C0180911201B3
:10096000909113012817390709F5C90133230CF4B5
:100970004F968C0115950795159507951595079533
:100980001595079515950795065F1F4F81E090E037
:10099000B8011ED380E090E06AEA0DD38AEA809322
:1009A0008401109383010093820104C030931301EA
:1009B000209312011F910F91089578941F920F9226
:1009C0000FB60F921124EF92FF920F931F932F9364
:1009D0003F934F935F936F937F938F939F93AF93C7
:1009E000BF93EF93FF93DF93CF93CDB7DEB72797F6
:1009F000F894DEBF7894CDBFA895E6E2F0E0808160
:100A00008068808382E487B980818064808380816C
:100A100086FDFDCF84B1898385B18A832A8139819E
:100A2000922F80E0830F911D9F838E838E819F8103
:100A3000899714F01C8202C081E08C8381E487B91D
:100A4000E6E2F0E0808180648083808186FDFDCFD6
:100A500084B1898385B18A834A8129818E819F816E
:100A600030E0281B390B942F80E0280F391F3F837B
:100A70002E8340911401509115018E819F81209108
:100A8000140130911501480F591F332314F42F5FBF
:100A90003F4FC901959587959A01281B390B3093D3
:100AA000150120931401809114019091150199234F
:100AB0000CF40196959587959F838E838E819F81F7
:100AC000409167005091680060911C018BDC8B8322
:100AD00086E487B9E6E2F0E08081806480838081EB
:100AE00086FDFDCF84B1898385B18A836A8189813E
:100AF000209165003091660040916500509166003C
:100B0000280F311D962F80E0280F391F552314F42C
:100B1000415E5F4FCA019595879595958795959507
:100B200087959595879595958795A901481B590BAC
:100B30005093660040936500809165009091660037
:100B400099230CF44F96959587959595879595954E
:100B5000879595958795959587959093680080934F
:100B60006700209167003091680080918201909128
:100B70008301821B930B0AF40196959587959093B8
:100B800068008093670080916700909168000D97DE
:100B900024F081E080931C0102C010921C0180911E
:100BA00067009091680088539F4F1CF481E0809308
:100BB0001C0180E487B91D828D81803108F046C018
:100BC000E6E2F0E004E210E00F2EF5E2EF2EFF2463
:100BD000F02D808180648083808186FDFDCFD801E7
:100BE0008C918983D7018C918A838A819981782F0E
:100BF00060E09B01290F311D30931B0120931A01E6
:100C0000409116015091170180911A0190911B019A
:100C10002091160130911701480F591F332314F406
:100C2000295F3F4FC901959587959595879595952E
:100C30008795DA01A81BB90BB0931701A093160191
:100C40008D818F5F8D838D81803118F2E6E2F0E037
:100C5000808180648083808186FDFDCF84B189831B
:100C600085B18A83E6E2F0E080818F77808380918E
:100C700016019091170199230CF407969595879585
:100C8000959587959595879590931901809318016F
:100C90008C81882341F081E08B838DE790E09093F5
:100CA0001B0180931A0180911A0190911B016B81A5
:100CB00092DC80911801909119016C814B8116DCB6
:100CC00080911C0181116EDC809184018A3A29F0A7
:100CD00080916500909166003EDE2796F894DEBF15
:100CE0007894CDBFCF91DF91FF91EF91BF91AF91FC
:100CF0009F918F917F916F915F914F913F912F9134
:100D00001F910F91FF90EF900F900FBE0F901F90CB
:100D1000189570D088F09F5790F0B92F9927B75148
:100D2000A0F0D1F0660F771F881F991F1AF0BA95AF
:100D3000C9F712C0B13081F077D0B1E0089574C026
:100D4000672F782F8827B85F39F0B93FCCF38695A5
:100D500077956795B395D9F73EF490958095709502
:100D600061957F4F8F4F9F4F0895E89409C097FB7F
:100D70003EF490958095709561957F4F8F4F9F4F72
:100D80009923A9F0F92F96E9BB279395F6958795B6
:100D900077956795B795F111F8CFFAF4BB0F11F479
:100DA00060FF1BC06F5F7F4F8F4F9F4F16C0882320
:100DB00011F096E911C0772321F09EE8872F762F56
:100DC00005C0662371F096E8862F70E060E02AF097
:100DD0009A95660F771F881FDAF7880F9695879583
:100DE00097F9089557FD9058440F551F59F05F3FEC
:100DF00071F04795880F97FB991F61F09F3F79F03D
:100E000087950895121613061406551FF2CF4695BE
:100E1000F1DF08C0161617061806991FF1CF869540
:100E20007105610508940895E894BB276627772724
:100E3000CB0197F9089566D008F48FEF08950BD091
:100E40009CC08DD028F092D018F0952309F07EC078
:100E500083C01124EACFC6DFA0F3959FD1F3950F8D
:100E600050E0551F629FF001729FBB27F00DB11D2E
:100E7000639FAA27F00DB11DAA1F649F6627B00DBE
:100E8000A11D661F829F2227B00DA11D621F739FA7
:100E9000B00DA11D621F839FA00D611D221F749FB5
:100EA0003327A00D611D231F849F600D211D822FFC
:100EB000762F6A2F11249F5750408AF0E1F0882343
:100EC0004AF0EE0FFF1FBB1F661F771F881F915050
:100ED0005040A9F79E3F510570F038C0A6CF5F3F44
:100EE000ECF3983EDCF3869577956795B795F79583
:100EF000E7959F5FC1F7FE2B880F911D969587950B
:100F000097F90895990F0008550FAA0BE0E8FEEF36
:100F100016161706E807F907C0F012161306E407BD
:100F2000F50798F0621B730B840B950B39F40A26B6
:100F300061F0232B242B252B21F408950A2609F494
:100F4000A140A6958FEF811D811D089597F99F6798
:100F500080E870E060E008959FEF80EC0895002441
:100F60000A941616170618060906089500240A940E
:100F700012161306140605060895092E0394000C94
:100F800011F4882352F0BB0F40F4BF2B11F460FF23
:100F900004C06F5F7F4F8F4F9F4F0895E199FECF41
:100FA0009FBB8EBBE09A99278DB30895A8E1B0E06E
:100FB00042E050E012C0262FE199FECF9FBB8EBBCE
:100FC0002DBB0FB6F894E29AE19A0FBE01960895F0
:100FD000F2DF272FF1CFDC01CB01FC01E199FECF3D
:100FE00006C0FFBBEEBBE09A31960DB20D924150A8
:0A0FF0005040B8F70895F894FFCFC1
:0A0FFA004604003200CC100A00008B
:00000001FF
